:020000040800F2
:1000000000040020E1010008450C0008450C000830
:10001000450C0008450C0008450C0008450C00087C
:10002000450C0008450C0008450C0008452A00084E
:10003000450C0008450C0008450C0008450C00085C
:10004000450C0008450C0008450C0008450C00084C
:10005000450C0008450C0008450C0008450C00083C
:10006000450C0008450C0008450C0008450C00082C
:10007000450C0008450C0008450C0008450C00081C
:10008000450C0008450C0008450C0008450C00080C
:10009000450C0008450C0008450C0008450C0008FC
:1000A000450C0008450C0008450C0008450C0008EC
:1000B00091230008450C0008450C0008450C000879
:1000C000450C0008450C0008450C0008450C0008CC
:1000D000450C0008450C0008450C0008450C0008BC
:1000E000450C0008450C0008450C0008450C0008AC
:1000F000450C0008450C0008450C0008450C00089C
:10010000450C0008450C0008450C0008450C00088B
:10011000450C0008450C0008450C0008450C00087B
:10012000450C0008450C0008450C0008450C00086B
:10013000450C0008450C0008450C0008450C00085B
:10014000450C0008450C0008450C0008312100084A
:10015000450C0008450C0008450C0008450C00083B
:10016000450C0008450C0008450C0008450C00082B
:10017000450C0008450C0008450C0008450C00081B
:10018000450C0008450C0008450C0008450C00080B
:10019000450C0008450C0008450C0008450C0008FB
:1001A000450C0008450C0008450C0008450C0008EB
:1001B000450C0008450C0008450C0008450C0008DB
:1001C000450C0008450C0008450C0008450C0008CB
:1001D000450C0008450C0008450C0008450C0008BB
:1001E00072B6374880F3098836484EF60851CEF289
:1001F0000001086040F20000CCF200004EF63471BD
:10020000CEF200010860BFF34F8FBFF36F8F40F253
:100210000000C0F2F0004EF68851CEF200010860F6
:10022000BFF34F8FBFF36F8F4FF00000E1EE100A66
:100230004EF63C71CEF200010860062080F314886F
:10024000BFF36F8F00F0E0FC02F0E2F84FF05530A2
:100250001D491E4A91423CBF41F8040BFAE71C4974
:10026000174A91423CBF41F8040BFAE719491A4A70
:100270001A4B9A423EBF51F8040B42F8040BF8E7C0
:1002800000201749174A91423CBF41F8040BFAE796
:1002900000F0BEFC02F0BEF8134C144DAC4203DA81
:1002A00054F8041B8847F9E700F03EF8104C114D54
:1002B000AC4203DA54F8041B8847F9E700F0A6BC07
:1002C00000080020000000080000002000040020BA
:1002D00000040020F834000800080020280800204E
:1002E00028080020301A0020E0010008E001000882
:1002F000E0010008E00100082DE9F04F2DED108A23
:10030000C1F80CD0C3689D46BDEC108ABDE8F08FE3
:10031000002383F311882846A047002000F096FEB2
:1003200000F030FE00DFFEE708B500F041FC0C4BAA
:100330007F21002219700F215A709A70DA701A7199
:100340005A719A71DA711A725A729972DA7200F0ED
:10035000F1FA41F2883000F077F800F045F8F8E75C
:100360002808002008B500F087FAA0F120035842C1
:10037000584108BD07B5054B02211B88ADF8043074
:1003800001A800F0C7FA03B05DF804FBBC31000817
:1003900010B51148C3680BB100F020FD0F4C104A96
:1003A0000D4800234FF47A7100F0DCFC236813B190
:1003B0002368013B2360636813B16368013B63609A
:1003C000084B1B7833B9636823B9022000F098FB0F
:1003D0003223636010BD00BF340800204C0D0020A4
:1003E000910300084808002038B5114C23680133F8
:1003F0001CD0104D104B2A689A4217D90F4B9B689E
:1004000003F1006303F580339A420FD2002000F01D
:10041000ABFA0B4B0220187000F064FB72B6094B6C
:100420001C6023682A6883F30888104738BD00BF22
:100430000000010804000108FFFF00082808002050
:100440004808002008ED00E02DE9F04FBC4B0546C0
:10045000BC489C680022C2608FB0202282F31188C1
:10046000C26898460AB100F0B9FC0023B64AB54804
:100470004FF47A7100F076FC002383F31188DFF8E3
:10048000E4920DB1C9F80050B04EC9F80430337091
:100490004FF0FF37012000F025FB002D00F0AF8169
:1004A000D9F80030002B40F0AA810FB0BDE8F08FE2
:1004B0000220FFF757FF00283AD1A54B1B88ADF863
:1004C0002430022109A800F025FAE3E74FF47A70FE
:1004D00000F0D2F9B0F1000BEFDB0220FFF742FF92
:1004E0000028EAD00BF1FF300428E6D8DFE800F05E
:1004F00003090E1114000EA8052340F8143D042131
:1005000001E08F48042100F005FA11E00421914830
:10051000F9E704219048F6E71C25284600F026FA62
:1005200004350990042109A800F0F4F92C2DF4D128
:1005300000F034FBFFF71EFF5FE10220FFF712FF20
:100540000028BAD0012000F00FFA0220307000F02D
:10055000C9FA4FF0000B5FFA8BFA504600F01CFA14
:100560000BF1010B044618B1504600F025FAF2E7F2
:1005700001230220337000F0A7FAD8F808309C421B
:1005800007D2204600F0F2F9013040F0198104341E
:10059000F3E700243470C9F80440C9E70220307042
:1005A00000F0A0FA322000F067F9B0F1000B84DB14
:1005B0001BF0030381D1D8F808100BEB04028A4228
:1005C0003FF67BAFBBF5807F3FF677AF634A9A4635
:1005D000DA4501920FDA4FF47A7000F04DF903908A
:1005E00003990029FFF669AF019A03990AF80210EE
:1005F0000AF1010AECE7C820FFF7B4FE00283FF437
:100600005CAF24B9554B4FF0FF321F681A60534B53
:100610002BF0030BA344A3EB040A5C4588D05AF8E3
:100620000410204600F0A8F9204600F09FF95AF87F
:100630000420904240F0C4800434EEE70220FFF72B
:1006400091FE00283FF439AF4FF0000B5D46D8F81B
:1006500008309B4534D2BBF1000F14D17A1C12D064
:1006600009973F494B689BB1002209A8135C6B4076
:10067000DBB2013251F82330042A83EA1525F5D183
:100680000BF1040BE3E7584600F070F90990E8E736
:100690001A46082012F0010F4FEA52021FBF82F0E3
:1006A0006D4282F4380282F4034282F02002013863
:1006B000F0D141F823200133B3F5807FE8D1D3E7AF
:1006C0000EA840F8285D1AE70EA8002340F8143D54
:1006D000642100F0FBF800287FF4EFAE0220FFF762
:1006E00041FE00283FF4E9AE099800F077F90EAB1F
:1006F00043F8240D0421184605E70EA8002340F80E
:10070000143D642100F0E2F800287FF4D6AE022008
:10071000FFF728FE00283FF4D0AE099800F06CF9EE
:100720000EAB43F8200DE5E70220FFF71BFE002883
:100730003FF4C3AE00F066F90EAB43F81C0DD9E7E9
:1007400028080020340800209103000848080020F1
:10075000BE3100082C080020300800204C08002082
:100760004C0900204C0D00200220FFF7FBFD002863
:100770003FF4A3AE09A9142000F04AF905460EA8DB
:10078000042140F8185D00F0C5F8294609A8BAE62A
:100790004FF47A70FFF7E6FD00283FF48EAE7B1C25
:1007A00005D1FFF7E7FD324800F056FC7DE63946FB
:1007B000002000F0E1F8002000F0D8F88742F0D0E7
:1007C0002C4B7BE60EA8002340F8143D642100F07A
:1007D0007DF800287FF471AE0220FFF7C3FD0028EA
:1007E0003FF46BAEFFF7C6FD41F2883000F034FCF9
:1007F000099800F007FA00F0D1F900254AE6002038
:1008000000F03AF80390039B002BFFF646AE012060
:1008100000F05AF9039B213B122B3FF63BAE01A29D
:1008200052F823F0B1040008CD0400083B0500088D
:100830009504000895040008950400089D0500082B
:10084000950400083D060008C9060008FB060008DC
:1008500029070008950400086907000895040008A6
:10086000910700083105000895040008C507000835
:10087000A0860100C031000837B5114A1278013254
:10088000D2B20024012A03468DF8074011D80D4842
:100890000268D5694FF47A7253430DF107010122C2
:1008A000A847012805D1084B9DF807001C7003B02C
:1008B00030BD4FF4FA7000F0CFFB4FF0FF30F6E799
:1008C00000080020D8100020580D002038B50E4B2D
:1008D0001A780132D2B2012A05460ED80B480368B5
:1008E000DC694FF47A734B4304222946A04704285D
:1008F00003D1074B0020187038BD4FF4FA7000F098
:10090000ABFB4FF0FF3038BD00080020D8100020AE
:10091000580D002030B4054C23689D69044B0A46ED
:10092000AC460146204630BC604700BFD8100020CE
:10093000A086010070B501F0FFFE094C094E207041
:10094000002530682378834208D901F0EFFE336830
:1009500005440133B5F5803F3360F2D370BD00BF6D
:10096000590D0020540D002001F09ABF00F10060E5
:1009700000F580300068704707B502AB00F10060F9
:1009800043F8041D0422194600F5803001F016FFDB
:1009900003B05DF804FB0000054B1A68054B1B789B
:1009A0001344834202D9104401F0C0BE00207047B6
:1009B000540D0020590D002038B5074D0446286815
:1009C000204401F0BBFE28B928682044BDE8384027
:1009D00001F0CCBE38BD00BF540D002010F0030361
:1009E00008D1B0F5007F05D800F10050A0F508400F
:1009F0000068704700207047014BC058704700BF27
:100A0000107AFF1F014B1868704700BF002004E0F8
:100A100070B52A4B1C68C4F30B03240C63B140F27D
:100A20001342934231D040F2194293422FD040F208
:100A3000214293422DD10323214A0C2505FB032398
:100A40005D6893F9082042F201039C4224D0B4F57A
:100A5000805F23D041F201039C4221D041F2030385
:100A60009C421FD041F207039C4208BF3122441E22
:100A70000C44013D0B46A3421ED215F9016F581CD0
:100A800096B1034600F8016CF5E70123D4E7022391
:100A9000D2E73F220B4DD6E73322E3E74122E1E7DD
:100AA0005A22E4E75922E2E72C2584421D7001D93D
:100AB000981C5A70401A70BD1846FBE7002004E0ED
:100AC000D0310008C4310008022804D14FF0804220
:100AD000034B9A6170470128FCD14FF00052F7E7B1
:100AE00000000240022804D14FF48042034B9A6177
:100AF00070470128FCD14FF40052F7E70000024094
:100B0000022805D1064A536983F480435361704734
:100B10000128FCD1024A536983F40053F6E700BF71
:100B20000000024010B50023934203D0CC5CC454B3
:100B30000133F9E710BD000010B501380A4410F97F
:100B4000013F3BB191F900409C4203D1914201D059
:100B50000131F4E791F90000181A10BD10B5013801
:100B600010F9013F0A462BB192F900409C4201F175
:100B70000101F5D092F90000181A10BD0246034693
:100B8000981A13F9011B0029FAD170470244034651
:100B9000934202D003F8011BFAE77047024B1A7820
:100BA000024B1A70704700BF580D0020000800204B
:100BB00038B5104D104C284600F010FB2146284651
:100BC00000F038FB23680D485A6DD2F8043843F022
:100BD0000203C2F8043800F03FFA0949206800F027
:100BE00041FC23685A6DD2F8043823F00203C2F89E
:100BF000043838BDD8100020CC33000840420F0024
:100C0000243400087047000070470000FEE7000031
:100C1000084A094B09498B4204D3094A00219342EF
:100C200005D3704752F8040F43F8040BF3E743F879
:100C3000041BF4E71C350008301A0020301A00208D
:100C4000301A00201EF0040F0CBFEFF30880EFF302
:100C500009808169004A1047610C00087047000054
:100C6000204B02681A60204B42681A601F4B826852
:100C70001A601F4BC2681A601E4B02691A601E4B35
:100C800042691A601D4B82691A601D4BC2691A6065
:100C90001C4B1D491A681D4B1A601A68120A0A700B
:100CA0001A681B4B1A701B4B1A681B4B1A601B4BA4
:100CB0001A681B4B1A601B4B1A681B4B1A601B4BA4
:100CC0001A681B4B1A601B4B1A681B4B1A601B4B94
:100CD0005A6A1B4B1A601B4B1B68DB0701D500BE11
:100CE000FEE7FEE78C0D0020900D0020980D0020FF
:100CF0009C0D0020940D0020800D0020840D00200C
:100D0000880D002028ED00E0640D0020680D002013
:100D1000780D00202CED00E0700D002030ED00E09B
:100D20006C0D00203CED00E05C0D002034ED00E097
:100D3000740D002038ED00E0600D002000ED00E0B3
:100D40007C0D0020F0ED00E0054B03F114025A6128
:100D50009A614FF0FF32DA6100221A62704700BFD9
:100D6000A00D0020F8B503614FF08043C2605C6ABB
:100D7000194B1A46022952F8145F38BF02219542D6
:100D800006461F460AD1586198611C62056045609D
:100D900081600819BDE8F84000F042BB186AAB68F2
:100DA000241A0C1902D3E41A2D6804E09C4202D2E2
:100DB000204400F043FBAB689C42F4D86B6873603E
:100DC00035601E606E60B460A9684FF0FF33091B88
:100DD000A960FB61F8BD00BFA00D002010B41B4C42
:100DE000234653F8141F814210D0416802680A60FC
:100DF000026851609A424FF00001C16003D09368CD
:100E000081680B4493605DF8044B70470A68626127
:100E100000209A425360C86003D15DF8044B00F093
:100E200007BB93688868034493604FF08042506A20
:100E3000226A821A9342E6D99B1A022B2CBFC01851
:100E400002305DF8044B00F0F9BA00BFA00D00209D
:100E5000024B00221B605B609A607047A00D00206F
:100E6000002303748268054B1B6899689142FBD28A
:100E70005A6803604260106058607047A00D0020FF
:100E800008B5202383F31188037C032B05D0042BA2
:100E90000DD02BB983F3118808BD436900221A6075
:100EA0004FF0FF334361FFF7DBFF0023F2E790E8E9
:100EB0000C001A6002685360F2E70000002303741C
:100EC0008268054B1B6899689142FBD85A68036099
:100ED0004260106058607047A00D0020054B1969F2
:100EE0000874186802681A6053601861012303745B
:100EF000FFF702BAA00D002030B54B1C87B00546A5
:100F00000A4C10D023690A4A01A8FFF72BFF284694
:100F1000FFF7E4FF049B13B101A8FFF75FFF23690C
:100F2000586907B030BDFFF7D9FFF8E7A00D0020E2
:100F3000810E000838B50C4D41612B6981689A68B3
:100F40009142044603D8BDE83840FFF789BF1846F0
:100F5000FFF786FF01232C61014623742046BDE87C
:100F60003840FFF7C9B900BFA00D0020044B1A6834
:100F70001B6990689B68984294BF002001207047CD
:100F8000A00D002010B5084C236820691A68226063
:100F90005460012223611A74FFF790FF0146206913
:100FA000BDE81040FFF7A8B9A00D002008B5FFF775
:100FB000DDFF18B1BDE80840FFF7E4BF08BD000041
:100FC0008260022202740022427482617047000033
:100FD0008368A3F1840243F8142C026943F8442C7B
:100FE000426943F8402C084A43F8242CC26843F86D
:100FF000182C022203F8102C002203F80F2C43F8BF
:10100000082CA3F1200070471103000808B5FFF772
:10101000DFFFBDE80840FFF723BF000010B5202325
:1010200083F31188FFF7D4FF00210446FFF782FF06
:10103000002383F31188204610BD0000024B1B697A
:1010400058610F20FFF74ABFA00D0020202383F333
:101050001188FFF7F3BF000008B50146202383F392
:1010600011880820FFF748FF002383F3118808BD8B
:1010700010B5054C2369036058610320FFF72EFF6C
:101080002369586910BD00BFA00D002003682BB173
:101090000022026059611846FFF7E2BE7047000067
:1010A00049B1064B42681B6918605A60136043607F
:1010B0000420FFF721BF4FF0FF307047A00D002044
:1010C0000368984206D01A68026050605961184659
:1010D000FFF7C6BE7047000038B504460D462068CD
:1010E000844200D138BD036823605C604561FFF72E
:1010F000B7FEF4E713B5446BD4F88C341A68117852
:10110000042916D1217A022913D1197912890123D0
:101110008B4013420DD101A904F1440001F0EEFD12
:10112000024630B1D4F88C44019B2179206800F04C
:10113000E5F902B010BD00000C3001F05DBD00000B
:101140004FF0FF330C3001F057BD0000443001F088
:1011500041BE00004FF0FF33443001F03BBE0000C1
:101160000C3001F02BBD00004FF0FF310C3001F0CE
:1011700025BD0000443001F00DBE00004FF0FF32ED
:10118000443001F007BE0000D0F88C2438B5136855
:1011900019780429054601D0012038BD017A0229B9
:1011A000FAD112795C89012090400440F4D105F114
:1011B0000C0001F0BDFC02460028EDD0D5F88C549F
:1011C0004FF480732868697900F086F9204638BDAD
:1011D000406BFFF7D9BF0000704700007FB50346A2
:1011E000114A43F8042B0125436002260F4B057278
:1011F00004460290019300F17C02294600964FF4C8
:1012000080730C3001F070FC094B0193029400963E
:101210004FF4807304F52172294604F1440001F073
:1012200049FD04B070BD00BF20320008D111000894
:10123000F51000080B68202282F311880A7903EB6D
:10124000820290614A79093243F822008A7912B108
:1012500003EB8203986102230372C0F88C1400230D
:1012600083F311887047000038B504460125022138
:10127000043001F0C3FB04F10C0025756FF001018F
:10128000FFF72AFF84F84C5004F144006FF001018D
:10129000BDE83840FFF720BF10B5012104460430F7
:1012A00001F0ACFB0023237584F84C3010BD000026
:1012B00038B5044600250C3001F02EFC04F1440042
:1012C000257501F00FFD201D84F84C50012101F01F
:1012D00095FB2046BDE83840FFF756BF90F84430F4
:1012E00003F06003202B19D190F84520212A0AD061
:1012F000222A4FF000030ED0202A0FD1084A826321
:101300000722C26304E0064B83630723C363002301
:101310000364012070478363C363F9E700207047CB
:1013200001080020D0F88C3437B51A6811780429E8
:1013300004461AD1017A022917D119791289012399
:101340008B40134211D100F14405284601F0A0FD65
:1013500058B101A9284601F0D1FCD4F88C44019B76
:1013600021790246206800F0C9F803B030BD0000C2
:1013700000EB8103F7B59C6905460E46F4B12023C6
:1013800083F3118805EB8607201D082101F036FB49
:10139000FB685B691B68443413B1204601F0BCFC58
:1013A00001A9204601F0AAFC024648B1019B314642
:1013B000284600F0A3F8002383F3118803B0F0BDA2
:1013C000FB685A691268002AF5D01B8A013B13405A
:1013D000F1D105F14402EAE7093110B550F8214096
:1013E000CCB1202383F311880421601801F006FB9F
:1013F000D4F88C241368527903EB820304F10C00B7
:10140000DB689B69596801F09DFB2046FFF7BCFE35
:10141000002383F3118810BD7047000000F0CCBF9B
:101420004FF08043002258631A610222DA6070474D
:101430004FF080430022DA60704700004FF0804395
:101440005863704700F09CBB012303700023436086
:10145000C36183620362C3624362036303814381A6
:101460007047000038B50446202383F31188002517
:101470004160C56005614561856100F093FB022311
:10148000237085F3118838BD70B500EB81030546E4
:101490005069DA600E46144618B110220021FFF799
:1014A00075FBA06918B110220021FFF76FFB3146D0
:1014B0002846BDE8704000F04DBC0000028902F0F3
:1014C00001020281428902F001024281002202618E
:1014D0004261826100F0D2BCF0B400EB8104478924
:1014E000E4680125A4698D403D43458123600023C4
:1014F000A2606360F0BC00F0EDBC0000F0B400EB53
:1015000081040789E468012564698D403D430581B4
:1015100023600023A2606360F0BC00F06BBD00009C
:1015200070B50223002504460370A0F84C5080F8E3
:101530004E5080F84F5005814581C5600561456179
:10154000856180F8345000F0A3FB63681B6823B109
:1015500029462046BDE87040184770BD43680278B0
:101560001B6880F85020052202700BB10421184737
:1015700070470000436890F850201B6802700BB160
:10158000052118477047000070B50023044680F815
:10159000343000F1440200F093FC63689B685BBB4D
:1015A00094F8445015F0600614D194F8453005F0D5
:1015B0007F0545EA0325B5F5407F00F0A58059D8A1
:1015C000022D00F0F1803FD8002D00F08780012D22
:1015D00000F0E4800021204600F0BCFE00212046FF
:1015E00000F0AEFE63681B6813B1062120469847E1
:1015F000062384F8343070BD204698470028CFD0A9
:1016000094F84B2094F84A3043EA0223E26B934269
:1016100038BFE36394F94430E56B002B4FF02003AF
:1016200080F20181002D00F0F080012284F8342046
:1016300083F311880021E36BA26B2046FFF75EFF66
:10164000002383F3118870BDB5F5807F4DD0B5F5CB
:10165000817FBFD194F84630002BBBD194F848303D
:1016600013F00F0126D01A06204640F1B78000F093
:1016700085FE1FE0B5F5C06F50D020D840F2023390
:101680009D4200F0AE80B5F5A06FA3D1B4F8443010
:10169000B3F5A06F0ED194F8463084F84E30204652
:1016A00000F04CFB63681B6813B10121204698478A
:1016B000032323700023A363E3632364A0E7B5F54A
:1016C000106F41D040F602439D4267D0B5F5006FE0
:1016D00080D104F14F03A363012333E004F14C03F1
:1016E000A3630223E36325648AE794F84630012B61
:1016F0007FF470AFB4F84C3023F00203A4F84C3000
:10170000A663E66326647BE794F84630012B7FF4FA
:1017100061AFB4F84C3043F00203EFE794F849208E
:10172000616894F848304D6894F8471043EA022302
:10173000204694F84620A84700283FF44BAF436862
:10174000A3630368E363DDE794F84F2094F8463021
:101750009A42AFD02378042B10D1202383F3118831
:101760002046FFF7ABFE86F31188636884F84F606C
:101770001B68032121700BB12046984794F846302E
:10178000002B97D084F84F300423237063681B68C4
:10179000002B8FD00221204698478BE72E4BA36366
:1017A0000223E363002388E794F8481011F0800FC8
:1017B000204601F00F010ED000F074FB012806D086
:1017C00002287FF407AF254BA363E0639AE7244B1D
:1017D000A363E56396E700F057FBEFE700F0C4FD75
:1017E00068E794F84630002B7FF4F4AE94F8483064
:1017F00013F00F013FF45EAF1B06204602D500F048
:10180000A9FD57E700F09CFD54E7032284F834203B
:1018100083F311882B462A4629462046FFF75CFEB3
:1018200085F3118870BD5DB1042284F8342083F300
:1018300011880021E36BA26B2046FFF74DFEFFE607
:10184000052284F8342083F311882B462A46294642
:101850002046FFF753FEE3E7483200084032000815
:101860004432000838B590F834300446062B22D8AC
:10187000DFE803F0370422373732370090F84B1097
:1018800090F84A20C36B42EA01229A4214D9C268F6
:10189000128AB3FBF2F502FB15356DB9202383F3F1
:1018A00011882B462A462946FFF728FE85F3118822
:1018B000022384F8343038BD032384F834302023E5
:1018C00083F3118800231A4619462046FFF704FEC9
:1018D000002383F3118838BD036C03B198470023BC
:1018E000E7E7002100F036FD0021204600F028FD4A
:1018F00063681B6813B10621204698470623D8E782
:1019000090F83420062A38B5044621D801239340A4
:1019100013F0670F1DD113F008050FD1DB0617D5A3
:10192000052380F83430202383F311882B462A4680
:101930002946FFF7E3FD85F3118838BDC3689B692D
:101940005B682BB9036C03B19847002384F83430EB
:1019500038BD002100F0FEFC0021204600F0F0FC24
:1019600063681B6813B10621204698470623EDE7FC
:10197000836D30B500229D68446D11464FF0FF30F5
:1019800004EB421301329542C3F80019C3F8101951
:10199000C3F80809C3F8001BC3F8101BC3F8080BF1
:1019A000EED24FF00113C4F81C3830BD890141F06C
:1019B0002001016103699B06FCD4122001F000B8EC
:1019C0002DE9F04F202387B00446456D83F311883D
:1019D00000F1640305934FF0000B2378012B04D032
:1019E000236E4BB96B69DB0606D4AB69059843F0EF
:1019F0001003AB61FFF73CFB8BF311884FF0000E37
:101A00004FF02009A36D9B685FFA8EF083421BD2D2
:101A1000202383F31188E0E7616D0A6A02F4F01372
:101A2000B3F5802F66D0B3F5402F0DD1C2F30A165F
:101A300002F00F0204EB820201F58051D3681F6AA5
:101A400000231A469E4248D1696911F01001E3D182
:101A5000012303FA00F2236E1A4200F08C8089F30E
:101A60001188AB6823F00103AB60236E23EA020305
:101A7000236681F3118804EB8003D3F80C80D8F837
:101A800014100B680093431C1B030293430104933F
:101A90004868009B98425FD2B8F81060676D1B1AC7
:101AA000B34228BF3346049EBE19D6F81869B6B2B1
:101AB000B3EB860F62D8029EBE1903968E6801961C
:101AC000A6F1040A9C46039E5AF8047F3760BCF1D5
:101AD000040F3BD9ACF1040CF5E713F0030F08BF7A
:101AE0000A68072B98BF3A7003F101039CBF120AE2
:101AF0000137A7E7C2F30A1602F00F0204EB8202D5
:101B000001F58051D3689B691F68D3F808805B6832
:101B1000A7EB030C00231F469E4208D1D3689969A6
:101B20008A684B68324433448A604B608CE713F018
:101B3000030F08BF0F689C4588BF88F8007003F149
:101B4000010384BF3F0A08F10108E5E7019E1E4436
:101B500003448E604B609BE7012189F31188AB68D9
:101B600043F00103AB6021B9D5F834381A43C5F806
:101B700034288BF311880EF1010E43E70021ECE7C6
:101B800010B5064C2046FFF75FFC4FF0A042002343
:101B90006265034A6366A265A36610BDE80D002076
:101BA0007032000870B50378012B86B005465BD112
:101BB0002F4B446D984213D12E4B5A6B42F080024A
:101BC0005A635A6942F080025A6100225A610E211A
:101BD000432001F07DF9284BE360284BC4F800381E
:101BE00000232B66C4F8003EC02323604FF4041387
:101BF000A3636E6D202000F0E3FE0123336133699F
:101C0000DB07FCD4122000F0DBFE3369002BFCDA8A
:101C10000026A6602846FFF7ABFE6B68C4F8106884
:101C2000DB68C4F81468C4F81C68FBB9144BA361E2
:101C30004FF0FF336361AB6E93B9124B009305F124
:101C40007003019305F536730293022303936846EC
:101C50000D4B04930595FFF7D9F9A866FFF7A6F990
:101C6000A36843F00103A36006B070BD074BDEE735
:101C7000E80D00200038024040140040030020021C
:101C8000003C30C07C320008C1190008083C30C05C
:101C9000F8B5446D054600212046FFF787FEA96D83
:101CA00000234FF001128F68C4F834384FF00066FB
:101CB000C4F81C284FF0FF3004EB431201339F425D
:101CC000C2F80069C2F8006BC2F80809C2F8080B34
:101CD000F2D20B68EB6563626B6D10221A611E69AC
:101CE00016F01006FBD1122000F06AFED4F800387E
:101CF00023F4FE63C4F80038A36943F4402343F09F
:101D00001003A3610923C4F81038C4F81438094B30
:101D1000EB60094BC4F8106BC4F8003BC4F81069C1
:101D2000C4F80039EB6D03F1100243F48013EA6547
:101D3000A362F8BD4C32000840800010426D90F85C
:101D40004E10D2F8003823F4FE6343EA0113C2F8C0
:101D5000003870472DE9F0410EB200EB86080D46C1
:101D6000D8F80C100F6807F00303022B50D0032B98
:101D700050D03D4A3D4F012B18BF1746446D4FEAE6
:101D8000451E04EB0E030022C3F8102B8A6905F1EF
:101D9000100C002A40D04A8A05F158035B013A43EF
:101DA000E2500123D4F81C2803FA0CF31343A64491
:101DB0004A69C4F81C380023CEF8103905F13F03F6
:101DC000002A39D00A8A898B9208012988BF4A43A0
:101DD000C16D04EB8303561841EA0242C6652946E9
:101DE0005A602046FFF7E2FDD8F80C301B8A43EA20
:101DF00085531F4305F148035B01E7500123D4F8E5
:101E00001C2803FA05F51543C4F81C58BDE8F081F9
:101E1000174FB3E7174FB1E704EB4613D3F8002B86
:101E200022F40042C3F8002BD4F81C28012303FA43
:101E30000CF322EA0303BAE704EB83030E4A5A6069
:101E400004EB461629462046FFF7B0FDD6F80039C8
:101E500023F40043C6F80039D4F81C38012202FAF2
:101E600005F523EA0505CFE7008000100080041087
:101E70000080081000800C1000040002826D1268BF
:101E8000C265FFF775BD00005831436D49015B58CD
:101E900013F4004004D013F4001F14BF01200220EB
:101EA000704700004831436D49015B5813F400400E
:101EB00004D013F4001F14BF01200220704700005B
:101EC00000EB8101CB68196A0B6813604B685360A3
:101ED0007047000000EB810330B5DD68AA69136824
:101EE000D36019B9402B84BF402313606B8A1468F8
:101EF000426D1C44013CB4FBF3F46343033323F011
:101F0000030302EB411043EAC44343F0C043C0F86B
:101F1000103B2B6803F00303012B09B20ED1D2F85A
:101F2000083802EB411013F4807FD0F8003B14BF57
:101F300043F0805343F00053C0F8003B02EB4112E2
:101F4000D2F8003B43F00443C2F8003B30BD000030
:101F50002DE9F041264D6E6D06EB40130446D3F893
:101F6000087BC3F8087B38070AD5D6F81438190758
:101F700006D505EB84032146DB6828465B68984755
:101F8000FA0733D5D6F81438DB072FD514B995F8EE
:101F900034305BB305EB8403D968CCB98B69488ACC
:101FA0005E68B6FBF0F200FB12628AB91868DA6864
:101FB00090420DD2121A83E81400202383F3118873
:101FC0000B482146FFF786FF84F31188BDE8F081B6
:101FD000012303FA04F26B8923EA02036B81CB68C5
:101FE00023B121460248BDE8F0411847BDE8F08121
:101FF000E80D002000EB810370B5DD68436D6C696E
:102000002668E6604A0156BB1A444FF40020C2F825
:1020100010092A6802F00302012A0AB20ED1D3F88D
:10202000080803EB421410F4807FD4F8000914BFB1
:1020300040F0805040F00050C4F8000903EB421219
:10204000D2F8000940F00440C2F80009D3F834087F
:10205000012202FA01F10143C3F8341870BD19B925
:10206000402E84BF4020206020682E8A841940F0D2
:102070000050013C1A44B4FBF6F440EAC440C6E701
:102080002DE9F041284C666D06EB40130546D3F868
:102090000879C3F80879F9071AD5D6F81038DA079D
:1020A00016D504EB8003D9684B691868DA6890424A
:1020B0002CD2121A4FF000081A60C3F804802023B3
:1020C00083F3118829462046FFF794FF88F311888F
:1020D0003B0619D5D6F83428012303FA05F5154235
:1020E00012D0202383F31188236E10482B432366DC
:1020F000D6F8343823EA0505C6F834580021FEF72F
:10210000C5FF002383F31188BDE8F081012303FAA2
:1021100005F2238923EA020323818B68002BD7D0A1
:10212000294620469847D3E7E80D00204C0E0020B2
:102130002DE9F74F8048446D6669A3691E4016F487
:10214000805F6661054608D000230366FFF7E8F963
:1021500003B0BDE8F04F00F087BC002E12DAD4F8CF
:10216000003E75489F071EBFD4F8003E23F00303CE
:10217000C4F8003ED4F8043843F00103C4F804382E
:10218000FFF7F8F9300504D500236B482B66FFF7FD
:10219000E5F9B1040CD5D4F8083813F0060FE3685C
:1021A00023F470530CBF43F4105343F4A053E36083
:1021B000320704D56B68DB680BB15F489847F302C0
:1021C0004ED4B7020CD5D5F85480DFF86CA10027A7
:1021D0004FF00109AB6D9B68F9B28B4280F08F80A4
:1021E000F5060DD5202383F31188A369534823F006
:1021F0001003A3610021FEF749FF002383F3118838
:102200003003D4F8184813D5E10302D50020FFF7B6
:102210009FFEA20302D50120FFF79AFE630302D5B9
:102220000220FFF795FE270302D50320FFF790FE5B
:1022300075038DD5E00702D50020FFF721FFA10728
:1022400002D50120FFF71CFF620702D50220FFF72D
:1022500017FF23077FF57CAF0320FFF711FF77E718
:10226000D5F854A0DFF8D4B04FF00009AB6D9B68EF
:102270005FFA89F7BB42A4D30AEB4713D3F80029CE
:1022800002F44022B2F5802F36D1D3F80029002A7B
:1022900032DAD3F8002942F09042C3F80029D3F88B
:1022A0000029002AFBDB3946686DFFF77FFB01231D
:1022B0002A89BB406FEA030808EA02022A8105EB7B
:1022C0008702D268926822B139461B480193904731
:1022D000019B202282F31188DAF8342808EA0202EE
:1022E000CAF834282A6E0021134358462B66FEF79D
:1022F000CDFE002383F3118809F10109B6E708EB4D
:102300004112D2F8003B03F44023B3F5802F10D1E3
:10231000D2F8003B002B0CDA6A8909FA01F322EAB1
:1023200003036B8105EB8103DB68DB680BB150466F
:10233000984701374EE700BFE80D00204C0E002003
:10234000436D03EB4111D1F8003B43F40013C1F896
:10235000003B7047436D03EB4111D1F8003943F462
:102360000013C1F800397047436D03EB4111D1F8F8
:10237000003B23F40013C1F8003B7047436D03EBAF
:102380004111D1F8003923F40013C1F80039704726
:102390004FF0804310B51A69920708D500241C61DC
:1023A000202383F3118800F0D1FA84F31188BDE86B
:1023B000104000F059BB00000E4A136C43F00103BB
:1023C00013640D4A936843F0010393604FF0804318
:1023D00053229A624FF0FF32DA6200229A615A6306
:1023E000DA605A6001225A6108211A601C2000F04C
:1023F0006FBD00BF00380240002004E0002070479D
:10240000FEE70000704700004FF0FF30704700000B
:1024100000F0A2BD08B500F055FB00F057FABDE88A
:10242000084000F001B9000070470000022906D002
:10243000032906D00129064818BF00207047054827
:102440007047032A9ABF044800EBC200002070477F
:1024500080340008343400080808002070B50446B1
:1024600008460D46FEF78AFBC6B2204601340378C3
:102470000BB9184670BD32462946FEF75DFB0028B1
:10248000F3D1012070BD00002DE9F04F07469BB04D
:1024900008460C461546FEF771FB3E49C6B220467B
:1024A000FFF7DCFF08B10736F6B23B492046FFF7DD
:1024B000D5FF08B11036F6B2632E01AE0CD8DFF8A6
:1024C000E480DFF8E4B0B14694F800A0BAF1000F60
:1024D0001CD189F800A003E02146304600F010FE30
:1024E0003046FEF74BFBC0B2431C5B0087E8280078
:1024F0002B7003236B70002302351946DAB2904229
:1025000005F102053ED81BB0BDE8F08FBAF1250FEA
:1025100032D120492046FEF721FB78B91F4A4946AF
:1025200002F10C0052F804EB41F804EB8242F9D1BD
:1025300012880A80073409F10E09C5E716492046BA
:10254000FEF70CFBC0B9164809F1020210F8011F92
:102550004FEA111E01F00F011EF808E011F80810F3
:1025600002F802EC584502F8011C02F10202EDD11A
:1025700009F118090834A7E789F800A0013409F126
:102580000109A1E7F25C05F8022C05F8011C0133F2
:10259000B4E700BFD4330008DC330008E53300089B
:1025A0000F7AFF1FF43300081B7AFF1F08B52023A2
:1025B00083F311880348FEF7B5FE002383F31188E7
:1025C00008BD00BFD810002010B50446052916D854
:1025D000DFE801F016150316161D202383F311887A
:1025E0000E4A0121FEF750FF20460D4A0221FEF758
:1025F0004BFF0C48FEF75CFE002383F3118810BDEF
:10260000202383F311880748FEF72EFEF4E72023EA
:1026100083F311880348FEF73FFEEDE7843300089B
:10262000A8330008D810002038B50C4D0C4C0D49CB
:102630002A4604F10800FFF727FF05F1CA0204F15A
:1026400010000949FFF720FF05F5CA7204F11800D0
:102650000649BDE83840FFF717BF00BF98150020B6
:10266000080800200834000812340008DC33000891
:10267000024AD368DB03FCD4704700BF003C024031
:1026800008B5094B1B7873B9FFF7F2FF074B1A69BE
:10269000002ABFBF064A5A6002F188325A601A689F
:1026A00022F480621A6008BDF6170020003C024048
:1026B0002301674508B50B4B1B7893B9FFF7D8FF8B
:1026C000094B1A6942F000421A611A6842F48052BA
:1026D0001A601A6822F480521A601A6842F4806202
:1026E0001A6008BDF6170020003C02400B2870B5A8
:1026F00013D80B4A0B4C137863B90B4E4FF00061A3
:1027000044F8231056F8235001330C2B2944F7D1F9
:102710000123137054F8200070BD002070BD00BF6D
:1027200028180020F8170020A0340008014B53F8A7
:1027300020007047A03400080C2070470B2810B50B
:10274000044601D9002010BDFFF7D0FF064B53F817
:1027500024300344984201D1012010BD0278FF2AA1
:10276000F0D10130F6E700BFA03400080B2810B507
:102770001AD8FFF77DFFFFF783FF0F49F324CC60E2
:10278000FFF776FFC300DBB243F4007343F00203AC
:102790000B610B6943F480330B61FFF769FFCB6872
:1027A00023B1CC60FFF786FF002010BDFFF782FF4A
:1027B000BDE81040FFF7C2BF003C02402DE9F047E2
:1027C000D40715464DD41318B3F1016F49D2324BDB
:1027D0001B68DA0745D5314CFFF752FFF323E3605E
:1027E000FFF746FF2F46401A40F20129032F884683
:1027F00001EB000618D8294C40F201197B1A43441A
:10280000012B01EB000623692FD823F0010323617C
:10281000FFF750FF2846BDE8F087366851F8043CC2
:10282000B34218D1043FE1E7B307E4D1236923F4AD
:1028300040732361236943EA090323610431D8F813
:1028400000303360BFF34F8FFFF712FFE368002BB8
:10285000E3D0F323E360236923F001032361FFF74F
:1028600029FF4FF0FF30BDE8F08723F44073236168
:10287000236943EA090323618A4631F8023B338026
:10288000BFF34F8FFFF7F4FE3688BAF80030B6B2C8
:10289000B342B3D0DFE700BF00380240003C024043
:1028A000084908B50B7828B153B9FFF7E9FE0123B1
:1028B0000B7008BD23B1BDE808400870FFF7FABEF1
:1028C00008BD00BFF6170020FEE7000010B5184C49
:1028D000FEF7BEFAFEF738FA00F0A4F88022154998
:1028E0002046FEF76DFB012344F8180C0374124BCD
:1028F000124AD96821F4E0610904090C0A4310491D
:10290000DA60CA6842F08072CA600E490A6842F012
:1029100001020A601022DA77202283F822200023A5
:1029200083F3118862B60848BDE81040FEF776BB15
:10293000C80D0020D034000800ED00E00003FA05C7
:10294000F0ED00E0001000E0D83400082DE9F84375
:102950001A4C4FF0804300256769586A04F1140847
:102960002E46226ABB68811A8B420CD961694145A7
:1029700022D013441B1A022B2CBFC0180230BDE812
:10298000F843FEF75BBD134423623B68D7F80C9015
:10299000C3F8048043456361FD6001D1FEF748FD43
:1029A00086F311883869C847202383F311884FF0D4
:1029B00080436769586AD4E7BDE8F883A00D00201A
:1029C000034B59685A68521A9042FBD8704700BFAF
:1029D000001000E083691943037C81610A2B03D155
:1029E0004369194205D170470B2B06D143698B43CC
:1029F00003D100234361FEF733BA704770B5046812
:102A000005460E46AC4200D170BDE3683343E36037
:102A100016B12269134203D0A1686068FFF7DAFF9C
:102A20002468EFE7034B044A1A60044B044A1A6017
:102A3000704700BF2C1A0020301A0020281A0020EE
:102A40000000022080B5074A536823F0010300AF5D
:102A50005360EFF30983683383F30988002383F31A
:102A6000118880BD30EF00E098B5202300AF83F3DC
:102A70001188104B5B6813F4006318D0F1EE103A24
:102A8000EFF309844FF0807344F84C3C0A4BDB6849
:102A900044F8083CA4F1680383F30988FEF766FA5A
:102AA00018B1064B44F8503C98BD054BFAE783F348
:102AB000118898BD00ED00E030EF00E02103000830
:102AC0002403000808B500F019FA064800F0CAFA15
:102AD000FEF7B8FCFEF780FBFFF7A6FCBDE8084058
:102AE000FEF79CBC8832000830B5039C01720433A9
:102AF00004FB0325C361049B03630021059B006065
:102B00004060C1604261026185610462426281622B
:102B1000C162436330BD00000022416A416101612E
:102B2000C2608262C2626FF00101FEF7D5BA000096
:102B300003694269934203D1C2680AB10020704719
:102B4000181D704703691960C2680132C260C2690A
:102B5000134482690361934224BF436A03610021E5
:102B6000FEF7AEBA38B504460D46E3683BB162697C
:102B7000131D1268A3621344E362002038BD237A58
:102B800033B929462046FEF78BFA0028EDDA38BD26
:102B90006FF00100FBE70000C368C269013BC3603E
:102BA0004369134482694361934224BF436A43618A
:102BB00000238362036B03B11847704770B520236D
:102BC000044683F31188866A3EB9FFF7CBFF0546BA
:102BD00018B186F31188284670BDA36AE26A13F81B
:102BE000015BA362934202D32046FFF7D5FF002387
:102BF00083F31188EFE700002DE9F74F1F460446E5
:102C00000E469146202383F311884FF0804800251B
:102C1000D8F82430FB18009307F1FF3AAB46A36ABB
:102C2000ABB91AF1030F06D939462046FFF79AFFD0
:102C300068B1002305E0D8F82410009A511A8F4299
:102C4000F3D283F31188284603B0BDE8F08FA16A60
:102C5000E36AA9EB05025B1A934228BF1346402B97
:102C60001CD9334601F1400251F8040B43F8040B20
:102C70009142F9D1A36A40334036A3624035A26A3B
:102C8000E36A9A4202D32046FFF786FF8BF311884E
:102C90004D45D8D2202383F31188C0E71A46304629
:102CA0000193FDF73FFF019BA26A1A441E44A262F2
:102CB0001D44E4E710B5029C0172043303FB0421B8
:102CC000C36100238362C362039B0363049B0060B0
:102CD0004060C46042610261816104624262436398
:102CE00010BD0000026AC260426A426102610022B5
:102CF0008262C2626FF00101FEF7EEB943690269B8
:102D00009A4203D1C2680AB100207047184650F8B1
:102D1000043B0B6070470000C368C2690133C360A5
:102D20004369134482694361934224BF436A436108
:102D30000021FEF7C5B9000038B504460D46E3682A
:102D40003BB123691A1DA262E2691344E3620020C9
:102D500038BD237A33B929462046FEF7A1F9002869
:102D6000EDDA38BD6FF00100FBE700000369196080
:102D7000C268013AC260C269134482690361934226
:102D800024BF436A036100238362036B03B11847C6
:102D90007047000070B5202304460E4683F3118867
:102DA000856A35B91146FFF7C7FF10B185F3118861
:102DB00070BDA36A1E70A36AE26A01339342A362E4
:102DC00004D3E16920460439FFF7D0FF002080F3E7
:102DD000118870BD2DE9F74F1F4604460D469146F8
:102DE000202383F311884FF080480026D8F8243040
:102DF000FB18009307F1FF3AB346A36AABB91AF187
:102E0000030F06D939462046FFF796FF68B1002325
:102E100005E0D8F82410009A511A8F42F3D283F3B8
:102E20001188304603B0BDE8F08FA06AE36AA9EBD1
:102E300006021B1A934228BF1346402B1CD905F1EA
:102E4000400355F8042B40F8042B9D42F9D1A36AA6
:102E50004033A3624036A26AE36A9A4204D3E1692E
:102E600020460439FFF782FF8BF311884E45D8D2F4
:102E7000202383F31188C0E71A4629460193FDF702
:102E800051FE019BA26A1A441D44A2621E44E2E75D
:102E9000026943699A4203D1C3681BB91846704757
:102EA0000023FBE7836A002BF8D0043B9B1AF5D084
:102EB0001360C368013BC360C3691A44836902613C
:102EC0009A4224BF436A0361002383620123E5E73A
:102ED00000F1604300F01F02400903F5614309015E
:102EE0008000C9B200F1604083F8001300F5614032
:102EF00001239340C0F8803103607047144B0021D8
:102F00001A694FF0FF321A61196158695A615961A3
:102F1000186A60F0805018621962586A5A625962E1
:102F20001A6C42F080521A640A4A106840F48070A9
:102F30001060186F00F44070B0F5007F1EBF4FF4B2
:102F4000803018671967536823F400735360704723
:102F50000038024000700040314B4FF080521A643C
:102F6000304A4FF4404111601A6842F001021A6081
:102F70001A689207FCD59A6822F003029A609A6850
:102F80009A60274B19469A6812F00C02FBD1186818
:102F900000F0F90018609A601A6842F480321A60F2
:102FA0000B689B03FCD54B6F43F001034B671C4B35
:102FB0005A6F9007FCD51C4A5A601A6842F080721A
:102FC0001A60184A53685904FCD5154B1A689201C7
:102FD000FCD5164A9A60164B1A68164B9A42164B45
:102FE0001AD1164A1168164A914215D140F20512BB
:102FF0001A600B4B9A6842F002029A609A6802F0DB
:103000000C02082AFAD15A6C42F480425A645A6E71
:1030100042F480425A66704740F20572E8E700BF0A
:10302000003802400070004008544007009488387F
:10303000002004E011640020003C024000ED00E0AC
:1030400041C20F414B6843608B688360CB68C360AB
:103050000B6943614B6903628B6943620B680360D0
:10306000704700001C4B0246186B10B540F2FF146D
:1030700020431863196D1948214319651146FFF75C
:10308000E1FF174802F11C01FFF7DCFF154802F1D0
:103090003801FFF7D7FF144802F15401FFF7D2FFC0
:1030A000124802F17001FFF7CDFF114802F18C01C7
:1030B000FFF7C8FF0F4802F1A801FFF7C3FF0E4852
:1030C00002F1C401FFF7BEFF0C4802F1E001BDE8C8
:1030D0001040FFF7B7BF00BF0038024000000240B9
:1030E0000004024000080240000C024000100240B0
:1030F0000014024000180240001C02400020024060
:1031000080EA0102844612F0030F4FD111F0030F41
:1031100032D14DF8044D11F0040F51F8043B0BD09F
:10312000A3F101329A4312F0803F04BF4CF8043BF4
:1031300051F8043B16D100BF51F8044BA3F1013202
:103140009A4312F0803FA4F101320BD14CF8043BBA
:10315000A24312F0803F04BF51F8043B4CF8044BEB
:10316000EAD023460CF8013B13F0FF0F4FEA33235C
:10317000F8D15DF8044B704711F0010F06D011F83B
:10318000012B0CF8012B002A08BF704711F0020F29
:10319000BFD031F8022B12F0FF0F16BF2CF8022B14
:1031A0008CF8002012F47F4FB3D1704711F8012B37
:1031B0000CF8012B002AF9D1704700BF121012132E
:1031C0001211000053544D3332463F3F3F00000080
:1031D00000000000C43100083F000000130400009C
:1031E000003200083F000000190400000A32000805
:1031F0003F00000021040000143200083F000000DE
:1032000053544D3332463430780053544D333246A4
:103210003432780053544D333246343436585800E3
:1032200055110008411100087D11000869110008BE
:1032300075110008611100084D11000839110008CE
:10324000000000000100000000000000000000007D
:1032500089150008651800080119000840004000A1
:10326000C0100020C010002001000000D01000207D
:103270008000000040010000030000007573625FE1
:1032800070756D70000000000000801600000000E6
:10329000AAAAAAAA00000000FF9F000000000000E8
:1032A00000A00A000000000000000000AAAAAAAACC
:1032B00000000000FFFF0000000000000000000010
:1032C0000000000000000000AAAAAAAA0000000056
:1032D000FFFF0000000000000000000000000000F0
:1032E00000000000AAAAAAAA00000000FFFF000038
:1032F00000000000000000000000000000000000CE
:10330000AAAAAAAA00000000FFFF00000000000017
:10331000000000000000000000000000AAAAAAAA05
:1033200000000000FFFF000000000000000000009F
:103330000000000000000000AAAAAAAA00000000E5
:10334000FFFF00000000000000000000000000007F
:10335000000000000A000000000000000300000060
:10336000000000000000000000000000000000005D
:10337000000000000000000000000000000000004D
:1033800000000000020000000000000071130008AF
:10339000D91300084000400068150020781500206F
:1033A0000200000000000000030000000000000018
:1033B000191400080000000010000000881500200B
:1033C000000000000100000000000000E80D0020E7
:1033D0000101020025424F41524425002553455228
:1033E00049414C25004D6174656B463430352D578D
:1033F000696E6700303132333435363738394142FF
:1034000043444546000000004172647550696C6F8A
:1034100074004D6174656B4634303557696E672DA5
:10342000424C0000C92500082D240008DD120008C8
:10343000AD250008430000003C34000809024300A9
:10344000020100C03209040000010202010005244B
:1034500000100105240100010424020205240600D5
:1034600001070582030800FF09040100020A0000A9
:10347000000705010240000007058102400000002E
:103480001200000088340008120110010200004000
:1034900083044057000201020301000004030904F1
:1034A000004000000040000000400000004000001C
:1034B0000000010000000200000002000000020005
:1034C00000000200000002000000020000000200F4
:1034D0006D61696E00000000F034000830180020B3
:1034E000281A002001000000C92800080000000080
:1034F00069646C6500000000FF0096000000000891
:10350000040000009C3400080000000000000000DF
:1035100000000000000000000000000000000000AB
:00000001FF
